:020000040000FA
:100200008A0183018B0181298A150C1900220C1B9C
:1002100036220B19BF228C1A7223730884007208CD
:0C0220008A00710E8300F00E700E0900C1
:100240000A14B401AF01B001B101B2010830B3002A
:100250002D0830210630B3002E0830218A01080015
:10026000AB0076102B1C5E2934086321AC000F39DB
:10027000AF070A302F02031C3F29AF0076142C0E63
:100280000F39B0077618B00A76100A303002031C16
:100290004B29B000761434087221AC000F39B10735
:1002A0007618B10A76100A303102031C5929B100C0
:1002B00076142C0E0F39B2077618B20AB40AAB0CBA
:1002C000B30B3129080082070134023404340834A6
:1002D00016343234643428345634123424344834D6
:1002E00096349234820700340034003400340034F1
:1002F00000340034013402340534103420344034E6
:10030000813403178D0183168C130C1483120C088F
:10031000F4000D0851228D0F8329031360308400EF
:100320008001840A041E9029A0308400803080005F
:10033000840A841D96298A15972BCD0ACD19CD01E3
:100340004D0ED500550DE039D300CE01CF01D001BF
:10035000D101D2014E08603E84000008D400530849
:10036000801F08384E044D220319E629D500D51BFD
:100370002822D800540DFE39D9002C225B08D51F45
:100380002022D51B24224E08033C031CE62994306E
:100390004E044D22D6005308D61F08384E044D2275
:1003A0000319E629D500D51B2822D800D61FDD2940
:1003B0000310D60DD6090314D60C0310560DD90020
:1003C0002C225B08D51F2022D51B2422CE0ACE1D4D
:1003D000AA29530810384D22D500D51F20222822E3
:1003E000D51B24225108CF025208031C520AD00206
:1003F000500803190C2AFF3A031D1B2ACF09CF0A04
:10040000530812384D222822D5004F025508031CEC
:100410004F08D500D517152A530811384D22D5009D
:100420004F025508031C4F08D5004D08683E840054
:10043000550880000800FF30CF00D01F0C2AFE298D
:10044000CF070318D00A0800D1070318D20A080002
:10045000DD00DD095D0A08000830D700DC01DA01A3
:10046000DB0159183A220310D80DDC0DD90CD70B3B
:10047000312A08005808DA070318DB0A5C08DB0792
:100480000800B900BA00BB00B90B442AB900BA0B86
:10049000442ABA00BB0B442A0800572200088313E1
:1004A00008005722740880008313F7140800F50031
:1004B0004030750203185E2AB030642A8317A030DA
:1004C0007502F030031CD03075078400080001303D
:1004D0007D2280307D2208000F393038B5008C2213
:1004E000350E0F39880007128716871587113508D2
:1004F0000F398800871587110800B5008C22350E4A
:100500000F398800071287128715871135080F39B0
:1005100088008715871108008316FF30880483122E
:10052000871207168715080E8711F039B70087154F
:10053000080887110F39B704B71B922A07128316D0
:10054000F030880583120800B6008A1577180A145F
:1005500000208A01B500FF30350603190800350870
:100560006E22360AA42A13304D22CB00CB08F71294
:10057000031DF716CA01CC013230A70033304D22DB
:10058000C2004218771667221424C0307D2215302D
:10059000A42276169D21F619DE2A7619D62AF61B94
:1005A000092B761B092B761A222BCA2A7611BC1F1F
:1005B000592B3C1D002BBC1D052BCA2AF611BD1A58
:1005C000E32A943041233D1AE72A94304D23BD1B82
:1005D000EB2A953041233D1BEF2A95304D233D18E2
:1005E000F32A96304123BD18F72A96304D23BD19C2
:1005F000FB2A973041233D19FF2A97304D23CA2A01
:10060000F71ECA2AF616F617B32AF612F613761351
:10061000C32AF613CF307D22761B1F2B4B0E0F39CA
:10062000031D152B20306E22162B6C224B086C22DA
:100630003A306E224A0E6C224A086C22CA2A2330B3
:10064000A422CA2A7612C8307D222B23771DCA2AFB
:1006500003306E22CA2A2408AD00AE0120213108E1
:10066000031D352B20306E22362B6C2230086C2275
:100670002E306E222F086C2220306E2256306E22D1
:100680000800C9007E30C7008330C60049084D22EB
:100690000E26F400490851220800C9007D30C70029
:1006A0008230C60049084D221426F4004908512220
:1006B00008003230C5009D21C5088A150319002D98
:1006C0008A017619D62AF619DE2A5B2B6722723048
:1006D000A422C0307D2213304D22C2000319892B81
:1006E000420E0F390319762B6C22782B20306E22A4
:1006F00042086C227C30A422D0307D2254306E22FD
:1007000068306E2272306E222D30771A2B306E22B6
:100710008B2B8A30A4229D2176198F2B8B2B76115F
:10072000BC1FCC2B3C1C9B2BBC1CAC2B3C1DC32BE3
:10073000BC1DC52B8B2BF612C20A42080F390A3A90
:10074000031DBB2B4208F039C2001030C207A03095
:1007500042060319C201BB2BF612C20342080F392D
:100760000F3A031DBB2B4208F939C200F93A031DA9
:10077000BB2B9930C2004208F712031DF716F40094
:1007800013305122662B7716C62B7712F401771A95
:10079000741433305122662B0D307D22C301672241
:1007A0009530A422C0307D22142410249D21761976
:1007B000DA2BD62B7611BC1F272CBC1DEC2B3C1D35
:1007C000E62B3C1CF32BBC1CFA2BD62BC30A103097
:1007D00043020318C301D52BC303103043020F306B
:1007E0000318C300D52B8030C7002030C600092471
:1007F0000E26012C7F30C7001F30C60009241426A6
:10080000012CF400430820244308033949045122F1
:10081000CF2B430820244308033949044D22080004
:10082000C03043077D220800C8014808202448083A
:10083000033949044D226E22C80A481E152C0800AF
:10084000C900C90C490E60391438C9000800C1013B
:10085000C301672285307714A42277104C30C11869
:1008600052306E2220306E220030411803306E224A
:100870000130411802306E22C0307D22A824C00011
:10088000C01B2822AD00AE0120212D30C01F2B300F
:10089000C008031920306E22F6103108031D542CB5
:1008A00020306E22F614552C6C223008031D5D2C6E
:1008B000F61C5D2C20306E225E2C6C222F086C22E0
:1008C00020306E2225306E22AC249D217619692CB1
:1008D000652C7611BC1FB32CBC1D752C3C1D752CD2
:1008E0003C1C792CBC1C8D2C642CC30A0130C30524
:1008F000642C03014306031D842C0430C700C60189
:1009000041080E26C1008C2C7E30C7008330C60003
:1009100040080E26C000A224292C03014306031D13
:10092000992C0330C700FF30C60041081426C100CF
:10093000A12C7D30C7008230C60040081426C000BC
:10094000A224292C4008F4009430410751220800C9
:10095000943041074D220800030143068030031DF7
:10096000C0307D220800C001C101C30167222930C7
:10097000A422400A6C22FC252C30A422C0307D2207
:1009800003014106031DC62C3330D02C0130410633
:10099000031DCC2C3D30D02C0230410603194730CA
:1009A000A422A625C200C21B2822AD00AE01202130
:1009B0002D30C21F2B30C208031920306E22F610D2
:1009C0003108031DE72C20306E22F614E82C6C222F
:1009D0003008031DF02CF61CF02C20306E22F12C78
:1009E0006C222F086C2220306E2225306E22BA2510
:1009F0009D217619FC2CF82C7611BC1F1A2EBC1DDB
:100A00000E2D3C1D082D3C1C152DBC1C532DF82C07
:100A1000C30A0B3043020318C301F72CC3030B3086
:100A200043020A300318C300F72C03014306031DD9
:100A3000202D0830C700C60140080E26C000522DE8
:100A400001304306031D2B2D0330C700C6014108AA
:100A50000E26C100522D02304306031D4B2D03010B
:100A60004106031D382D7E30C7008330C600482D57
:100A700001304106031D402D7E30C700C601482DC0
:100A800002304106031DB62C0130C7008330C6007A
:100A900042080E26942D8030C7002030C600AE25B7
:100AA0000E269D2DB62C03014306031D5F2D073036
:100AB000C700FF30C60040081426C000932D013047
:100AC0004306031D6B2D0230C700FF30C6004108EE
:100AD0001426C100932D02304306031D8C2D030103
:100AE0004106031D782D7D30C7008230C600892D58
:100AF00001304106031D812D7D30C700FF30C60047
:100B0000892D02304106031DB62C0030C70082300B
:100B1000C60042081426942D7F30C7001F30C6003F
:100B2000AE2514269D2DB62CF400400EC800480DAD
:100B3000E039103841045122B62CF400400EC800B0
:100B4000480DE039183844045122B62C400EC80034
:100B5000480DE039103841044D22080003304302AB
:100B6000C400400EC800480DE03918384404C400E1
:100B70004D22080003014306031DC02D8030FA2DCD
:100B800001304306031DC62DC030FA2D0230430646
:100B9000031DCC2DCC30FA2D03304306031DD22D7E
:100BA0008430FA2D04304306031DD82D8530FA2DEC
:100BB00005304306031DDE2D8630FA2D0630430630
:100BC000031DE42D8730FA2D07304306031DEA2D5F
:100BD0008830FA2D08304306031DF02D8930FA2D98
:100BE00009304306031DF62D8A30FA2D0A304306DC
:100BF00003198B307D22080022306E220830C80095
:100C0000400EF400740DE0391838F4004D226E22C5
:100C1000740AC80B052E22306E220800C800480A4C
:100C2000C706031946080800C8004803C60603198A
:100C300047080800C001C101C30167224119372ECE
:100C4000C118342E5D30A42206306E2220306E2270
:100C500041182F2E0030C11901306E22502E033062
:100C6000C11902306E22502E6330A422242E410876
:100C70000739073A03194A2E07306E2220306E22B8
:100C8000410A03396C2220306E220430C11905302C
:100C90006E22502E6A30A4220330C11902306E2217
:100CA0005130A422C0307D222930A422400A6C2277
:100CB000FC253A306E22FE26C200C21B2822AD005F
:100CC000AE0120212D30C21F2B30C2080319203065
:100CD0006E22F6103108031D712E20306E22F6149C
:100CE000722E6C223008031D7A2EF61C7A2E2030CC
:100CF0006E227B2E6C222F086C2220306E22253033
:100D00006E2205279D217619862E822E7611BC1D16
:100D1000992E3C1D932E3C1CA02EBC1CCA2EBC1B25
:100D2000822E8A156B2DC30A033043020318C301B8
:100D3000812EC3030330430202300318C300812E07
:100D400003014306031DB22E1030C700C601410D3A
:100D50000E39C11901380E26C1000310C10C031849
:100D6000C115C92E01304306031DBD2E0830C70032
:100D7000C60140080E26C000C92EBC1BC22E420868
:100D80001727C82E7E30C7008330C60042080E26C3
:100D9000F62E1D2E03014306031DDD2E0F30C70066
:100DA000FF30C600410D0E39C11901381426C100AB
:100DB0000310C10C0318C115F52E01304306031DA5
:100DC000E92E0730C700FF30C60040081426C000D7
:100DD000F52EBC1BEE2E42082027F42E7D30C700D6
:100DE0008230C60042081426F62E1D2EF400400E56
:100DF000C800480DE039410451221D2E400EC800A4
:100E0000480DE03941044D22080003014306031D4B
:100E10000B2F8030152F01304306031D112FC030DA
:100E2000152F023043060319D1307D220800C80077
:100E3000313C031832344808633C031864340034EE
:100E4000C8009C3C031800344808CE3C03189C346E
:100E5000CE34C001672247307714A4227710C03007
:100E60007D22400AAD00AE0120213008031D3B2F3A
:100E700020306E223C2F6C222F086C2220306E22F4
:100E800072279D217619452F412F7611BC1FB32A59
:100E90003C1D5C2F3C1C4F2FBC1C552F412FC00A02
:100EA000103040020318C0012A2FC0031030400246
:100EB0000F300318C0002A2FC8014008103803174C
:100EC0008F00031348088327F40048085122C80FF5
:100ED000622FF714672254307714A42277104F3012
:100EE0004122B32A4008103803178F000313C801AA
:100EF0004808202448080339490483276E22C80A79
:100F0000481E782F080003178D0083168C170C14C9
:100F10000000000083120C0803130800C0016722C0
:100F200061307714A4227710C0307D22400AAD00D2
:100F3000AE0120213008031DA02F20306E22A12FEA
:100F40006C222F086C2220306E2272279D21761988
:100F5000AA2FA62F7611BC1FB32A3C1DC12F3C1C03
:100F6000B42FBC1CBA2FA62FC00A103040020318A1
:100F7000C0018F2FC003103040020F300318C00093
:100F80008F2FC8014008103803178F00031348083B
:100F90004D22F400480883277406031DD927C80F83
:100FA000C72F672273307714A42277104F30412265
:100FB000B32AFC30C805480803178D0003134D22DF
:100FC00003178C008E0183168C170C158B1355306C
:100FD0008D00AA308D008C14000000008B170C11BE
:100FE0000313831248080339033A03190800C80A97
:020FF000DB2FF5
:1010000082075434723461346E3473346D3469340D
:101010007434743465347234203476346534723404
:101020002E34203432342E343834FF344234613498
:1010300074347434653472347934FF34543469341C
:101040006D3465347234FF34543469346D3465342E
:101050002134FF3443346834FF342034533465344E
:10106000743455347034FF34433465346E3474341E
:10107000653472343A3420342034FF344D346134D2
:10108000783469346D3475346D343A342034FF3437
:101090004D3469346E3469346D3475346D343A349A
:1010A0002034FF34203449346E3466346C34753463
:1010B00065346E34633465342034FF344C34653425
:1010C000663474342034FF345234693467346834FD
:1010D00074342034FF3453347734693474346334D3
:1010E00068342034FF345334653474342034543439
:1010F00069346D3465347234FF3420344D346934CE
:101100006E3420343A342034303430342034533484
:1011100065346334FF344E346F34743420344134D6
:1011200063347434693476346534FF34533465344D
:10113000743420344D346F34643465346C3420346A
:101140004E3461346D346534FF3453346134763455
:101150006534203454346F342034453445345034AD
:1011600052344F344D3420343F34FF3459344534F5
:1011700053342D34013420347C3420344E344F34F5
:101180002D344D3465346E347534FF34533461344A
:10119000763465346434203454346F342034453428
:1011A0004534503452344F344D34FF3450346F345E
:1011B00077346534723420344F3446344634203426
:0811C000213421342134FF34F5
:10120000FF345334773469347434633468342034AD
:101210004F344634463420344D346F3464346534AE
:101220006C342134FF3446344C3441345334483424
:1012300020344F347034653472346134743469341A
:101240006F346E347334FF3445344E345434453483
:1012500052342D34013420347C342034513455340C
:10126000493454342D344D3465346E347534FF3480
:101270004C346F34613464342D34013420347C3484
:10128000203453346134763465342D340034FF34E3
:101290004C346F346134643420344D346F346434EE
:1012A00065346C342D340134FF344D346F34643480
:1012B00065346C3420344C346F34613464346534B8
:1012C0006434FF344F347634653472347734723496
:1012D00069347434653420344D346F346434653487
:1012E0006C342D340134FF344D346F346434653440
:1012F0006C3420344F34763465347234773472343D
:1013000069347434743465346E34FF345434723454
:1013100069346D34203442347534743474346F3429
:101320006E3473342034FF34443453344334FF3444
:10133000023406340F341F340F34063402340034C0
:1013400008340C341E341F341E340C34083400347A
:1013500004340E341F340E340E340E340E34003484
:101360000E340E340E340E341F340E340434003474
:10137000003417341F341C341E340034003400345D
:1013800000341D341F3407340F340034003400346B
:1013900000340E340E3404340E3411341F3400344F
:1013A000003400340E341534113411340E3400344A
:0213B000FF3408
:101400000C11A10A12302106031D0B2AA101101094
:101410008E018F010800211C132A08309700B83074
:10142000A201302208001F15093097000430A200E5
:10143000AE303022A201210CA0002003683E8400BF
:1014400000087F39A000A00DA20D200DA20DFC39CF
:10145000801F302A9502031C96032208960208007A
:1014600095070318960A2208960708000C1383169E
:101470001E088312A3009E0CA30C9E0CA30C1F0D30
:10148000A000200E0739A03E84000008DE000408FA
:101490000739603E8400673A03199B220408633AC7
:1014A0000319A92223087F39A31F9522800004086D
:1014B000633C031C682A7713801B77177F308005F5
:1014C0000310000C80077F30801B8000771B801783
:1014D000081F8F2ADE1B7E2ADE09DE130008A30008
:1014E000A31F772A5E070318FF3080008F2A5E084B
:1014F000800203188F2A800980178F2ADE130008C4
:10150000A300A31B892ADE075E08DE1B7F30800054
:101510008F2A5E088002801B8F2A800980131F0893
:10152000083E413879399F0008000310A30DA30934
:101530000314230C08002308A400771125082402B3
:10154000031C77158030081AFF30881A0030A3007A
:101550000800771E0800F71E0800761B0800230805
:10156000403C031CB72AF61E0800F612BA2AF61AE7
:101570000800F6161F309B000230A80008000B116F
:101580000E308600060E0F39BE000D3086000608AC
:10159000F039BE040B308600060E0F39BF0007304D
:1015A00086000608F039BF043C083E06031D761588
:1015B000BE00BC063D083F06031DF615BF00BD0674
:1015C0003C083D05FF3A0319F7113E093C04FF3A78
:1015D000031DEF2A3F093D04FF3A0319F72A1F3084
:1015E0009B000530A800F715AA013030A900A60B12
:1015F00008000930A6009601FF30950009309700D9
:101600001014C508031DC503F71D1A2BBC1F1A2B88
:10161000A90B1A2B7615F6151F309B000230A80077
:101620000830AA1904302A1A0430AA1A0230A90074
:10163000AA1EAA0AA8080319202BA80B202B9B017D
:10164000761F262B1F30271A03019B00771D2E2B98
:10165000051A2E2B1F30A71A03019B00A70B0800A9
:101660003230A7007616F61E0800F617CA030319D3
:10167000692B4A080F390F3A031D08004A08F93947
:10168000CA00F93A031D0800F71E4A2B1F309B00C1
:101690000230A8005930CA00CB034B080F390F3A6B
:1016A000031D08004B08F939CB00F93A031D080067
:1016B0005930CB00CC034C080F390F3A031D0800FA
:1016C0004C08F939CC00F93A031D08002330CC004E
:1016D0000800CC08031D0800CB08031D0800F61203
:1016E000761708009818932B1819932B1A08DE0008
:1016F000F03A0319912B83175F080739C43E840021
:1017000084191C3E84000008831384008030041E6A
:10171000DE0004080739A03E84005E088000DF0A6E
:101720000800DF0108001A081812181608008A01BC
:10173000850186018701880189018316FF308500B4
:10174000F030860080308700F03088000730890054
:10175000423081008C018D010C150C178C168030E5
:101760009F00831241309F00073092009B010F3091
:101770009D00F601F701A101CD015D30A5007616AF
:10178000A8018316243098000B3099008312903002
:1017900098001930412203308800871587110F30D7
:1017A00041228715871105304122871587110230A4
:1017B00088008715871128307D220C307D22063065
:1017C0007D2240307D2297307714A422771081014A
:1017D0000B118B160B178B17051E07146722003091
:1017E000A42283163E30920083121F309B001F30CC
:1017F0004122831631309200831218309B001F3033
:10180000412283162A309200831215309B001F302C
:10181000412283161F30920083120F309B00233029
:10182000412283163E30920083129B01B32A031794
:101830008D0183168C138C181B2C0C1483120D082D
:101840008A014D228A158C060319322C8C008316CE
:101850000C158B1355308D00AA308D008C148B170E
:0E1860000C1183128D0F192C0313F7100800C2
:101A00008A016722D530A422C0307D22B530A422BD
:101A10008A019D218A1576190E2D082D76118A01CD
:101A2000BC1F662B8A153C1D162D082D3230C500B3
:101A3000F7118A019D21C5088A150319222D7619EF
:101A40000E2D192DF71C3D2D8A016722A430A422EA
:101A5000C0307D22B530A4228A157619302D2D2D67
:101A60007611BC1F3D2D3C1D362D2D2D17248A01CE
:101A70006722C530A4225F3041228A0167220030EC
:101A80007714A422771083161F30920083120F3030
:101A90009B001F30412283162A309200831215309A
:101AA0009B001F3041228316313092008312183080
:101AB0009B001F30412283163E30920083121F305C
:101AC0009B001F3041229B017F304122672207107B
:101AD0006F3041228129C001C3018A0167229330FE
:101AE0007714A42251307710A422C0307D222930EF
:101AF000A422400A6C224008D43E40191C3E4D22CC
:101B0000C1002B30411E2D306E2220306E2201305C
:101B10006E2220306E228A154119AE2DC118A92DD2
:101B20008A015D30A4228A0106306E2220306E22A6
:101B30008A154118A22D8A0100306E2201306E22D2
:101B40008A15CA2D8A0103306E2202306E228A1550
:101B5000CA2D8A016330A4228A15932D41080739C2
:101B6000073A0319C32D8A0107306E2220306E22F6
:101B7000410A03396C2220306E2204306E22053077
:101B80006E228A15CA2D8A016A30A42203306E2281
:101B900002306E228A1518268A019D218A1576192F
:101BA000D22DCC2D7611BC1DE42D3C1DDE2D3C1C10
:101BB000EB2DBC1CFD2DBC1BCC2D2C2EC30A0330E1
:101BC00043020318C301CA2DC3030330430202308A
:101BD0000318C300CA2D03014306031DF32DC00AD9
:101BE0000730C0056D2D01304306031DF92D411648
:101BF0000E2EC10A1730C1050E2E03014306031D28
:101C0000052EC0030730C0056D2D01304306031DAE
:101C10000B2E41120E2EC1031730C1054108F400EE
:101C20004008D43E40191C3E8A0151228A156D2D70
:101C300003014306031D1E2EC030282E013043062B
:101C4000031D242EC330282E023043060319C7304B
:101C50008A017D228A1508008A010C307D226722C4
:101C6000A430A422C0307D22B530A4228A019D2157
:101C70008A1576193C2E362E7611BC1F4A2E3C1D35
:101C8000422E362E17248A016722C530A4224F30F7
:101C90004122B32A8A01672212307714A4227710D6
:101CA000C0307D2223307714A42277108A019D2131
:101CB0008A1576195C2E562E76113C1D632EBC1BA0
:101CC000562E8A01B32A8A01672212307714A42281
:101CD0007710C0307D2237307714A42277108A0124
:101CE0009D218A157619752E6F2E8A0176113C1D5D
:0E1CF000292FBC1D8E2FBC1FB32A8A156F2E04
:1020000000340034003400349C3400340034003494
:1020100000340034003400346434003400340034BC
:1020200000347D348334003456346534743472346F
:102030004E3443342034313420342034203420349E
:1020400000349C3400340034003400340034003454
:10205000003464340034003400340034003400347C
:1020600000347D348334FF346F346E3420342034B4
:102070005634793473346B346F3476346B34613462
:102080000034003400349C34003400340034003414
:10209000003400340034643400340034003400343C
:1020A00000347D348334FF34203420342034203411
:1020B00050346C3479346E3420342034203420345D
:1020C000003400349C3400340034003400340034D4
:1020D00000340034643400340034003400340034FC
:1020E00000347D348334FF342034203420342034D1
:1020F00053346D34653472346F3476346B346134F8
:10210000003400340034003400349C340034003493
:1021100000340034003400340034643400340034BB
:1021200000347D348334FF34003400340034003410
:102130004E3443342034323420342034203420349C
:102140000034003400340034003400349C34003453
:10215000003400340034003400340034643400347B
:1021600000347D348334FF34FF34FF34FF34FF34D4
:102170004E3443342034333420342034203420345B
:1021800000340034003400340034003400349C3413
:10219000003400340034003400340034003464343B
:1021A00000347D348334FF3413341034113412344A
:1021B0004E3443342034343420342034203420341A
:1021C000003400340034003400340034003400346F
:1021D000003400340034003400340034003400345F
:1021E00000347D348334FF3404340534063407343A
:1021F0004E344334203435342034203420342034D9
:10220000003400349C340034003400340034003492
:1022100000340034643400340034003400340034BA
:1022200000347D348334003456346534743472346D
:102230004B3472346934643465346C342E344C3429
:1022400000349C3400340034003400340034003452
:10225000003464340034003400340034003400347A
:1022600000347D348334FF346F346E3420344B3487
:102270005634793473346B346F3476346B34613460
:102280000034003400349C34003400340034003412
:10229000003400340034643400340034003400343A
:1022A00000347D348334FF347234693464346534EB
:1022B00050346C3479346E3420342034203420345B
:1022C0009C340034003400340034003400340034D2
:1022D00064340034003400340034003400340034FA
:1022E00000347D348334FF346C346B3461342034F7
:1022F00053346D34653472346F3476346B346134F6
:1023000000340034003400349C3400340034003491
:1023100000340034003400346434003400340034B9
:1023200000347D348334FF3400340034003400340E
:102330004E3443342034313420342034203420349B
:102340000034003464340034003400340034003489
:10235000003400349C340034003400340034003441
:1023600000347D348334FF34FF34FF34FF34FF34D2
:102370004B3472346934643465346C342E345234E2
:10238000003400340034003400349C340034003411
:102390000034003400340034003464340034003439
:1023A00000347D348334FF34133410341134123448
:1023B0004E3443342034323420342034203420341A
:1023C0000034003400340034003400349C340034D1
:1023D00000340034003400340034003464340034F9
:1023E00000347D348334FF34043405340634073438
:1023F0004E344334203433342034203420342034D9
:10240000003400349C340034003400340034003490
:1024100000340034643400340034003400340034B8
:1024200000347D348334003456346534743472346B
:102430004B3472346934643465346C342E344C3427
:102440009C349C34003400340034003400340034B4
:102450006434643400340034003400340034003414
:1024600000347D348334FF346F346E34203456347A
:102470005634793473346B346F3476342E344C34B0
:102480000034003400349C34003400340034003410
:102490000034003400346434003400340034003438
:1024A00000347D348334FF3420346B347234693427
:1024B00050346C3479346E34203420342034203459
:1024C00064349C340034003400340034003400346C
:1024D0009C3464340034003400340034003400345C
:1024E00000347D348334FF3464346C346F342034EE
:1024F0005634793473346B346F3476342E3452342A
:1025000000340034003400349C340034003400348F
:1025100000340034003400346434003400340034B7
:1025200000347D348334FF3400340034003400340C
:102530004E34433420343134203420342034203499
:102540000034003464340034003400340034003487
:10255000003400349C34003400340034003400343F
:1025600000347D348334FF34FF34FF34FF34FF34D0
:102570004B3472346934643465346C342E345234E0
:10258000003400340034003400349C34003400340F
:102590000034003400340034003464340034003437
:1025A00000347D348334FF34133410341134123446
:1025B0004E34433420343234203420342034203418
:1025C0000034003400340034003400349C340034CF
:1025D00000340034003400340034003464340034F7
:1025E00000347D348334FF34043405340634073436
:1025F0004E344334203433342034203420342034D7
:10260000003400349C349C340034003400340034F2
:102610000034003464346434003400340034003452
:1026200000347D3483340034563465347434723469
:102630004B3472346934643465346C342E344C3425
:1026400000349C340034003400340034003400344E
:102650000034643400340034003400340034003476
:1026600000347D348334FF346F346E34203473345B
:102670005634793473346B346F3476346B3461345C
:102680000034003400349C3400340034003400340E
:102690000034003400346434003400340034003436
:1026A00000347D348334FF342034623472347A341D
:1026B00050346C3479346E34203420342034203457
:1026C0009C340034003400340034003400340034CE
:1026D00064340034003400340034003400340034F6
:1026E00000347D348334FF3464346F3475342034E3
:1026F00053346D34653472346F3476346B346134F2
:1027000000340034003400349C340034003400348D
:1027100000340034003400346434003400340034B5
:1027200000347D348334FF3400340034003400340A
:102730004E34433420343134203420342034203497
:102740000034003464349C340034003400340034E9
:10275000003400349C3464340034003400340034D9
:1027600000347D348334FF34FF34FF34FF34FF34CE
:102770004B3472346934643465346C342E345234DE
:10278000003400340034003400349C34003400340D
:102790000034003400340034003464340034003435
:1027A00000347D348334FF34133410341134123444
:1027B0004E34433420343234203420342034203416
:1027C0000034003400340034003400349C340034CD
:1027D00000340034003400340034003464340034F5
:1027E00000347D348334FF34043405340634073434
:1027F0004E344334203433342034203420342034D5
:10280000003400349C34003400340034003400348C
:1028100000340034643400340034003400340034B4
:1028200000347D34833410344D346F3474346F3459
:102830004B3472346934643465346C342E344C3423
:1028400000349C340034003400340034003400344C
:102850000034643400340034003400340034003474
:1028600000347D348334FF3472342E3420346C349D
:102870005634793473346B346F3476346B3461345A
:102880000034003400349C3400340034003400340C
:102890000034003400346434003400340034003434
:1028A00000347D348334FF346534743461346434EB
:1028B00050346C3479346E34203420342034203455
:1028C0009C340034003400340034003400340034CC
:1028D00064340034003400340034003400340034F4
:1028E00000347D348334FF346C346F34203420342E
:1028F00053346D34653472346F3476346B346134F0
:1029000000340034003400340034003400349C348B
:1029100000340034003400340034003400346434B3
:1029200000347D348334FF34003400340034003408
:1029300050346F34643476346F347A3465346B34A5
:102940000034003464340034003400340034003483
:10295000003400349C34003400340034003400343B
:1029600000347D348334FF34FF34FF34FF34FF34CC
:102970004B3472346934643465346C342E345234DC
:10298000003400340034003400349C34003400340B
:102990000034003400340034003464340034003433
:1029A00000347D348334FF34133410341134123442
:1029B0004E34433420343334203420342034203413
:1029C0000034003400340034003400349C340034CB
:1029D00000340034003400340034003464340034F3
:1029E00000347D348334FF34043405340634073432
:1029F0004E344334203434342034203420342034D2
:102A00009C3400340034003400340034003400348A
:102A100064340034003400340034003400340034B2
:102A200000347D3483340534563472347434753450
:102A30004E3461346B346C346F346E3420344C3427
:102A400000349C340034003400340034003400344A
:102A50000034643400340034003400340034003472
:102A600000347D348334FF346C346E3469346B3419
:102A700050347234653464346B346C346F346E3477
:102A8000003400349C34003400340034003400340A
:102A90000034003464340034003400340034003432
:102AA00000347D348334FF3420343234783453346A
:102AB0004F347434613463346B34793420342034CB
:102AC0000034003400349C340034003400340034CA
:102AD00000340034003464340034003400340034F2
:102AE00000347D348334FF346534723476346F348B
:102AF00056347234743475346C346B34613420342D
:102B000000340034003400349C3400340034003489
:102B100000340034003400346434003400340034B1
:102B200000347D348334FF34003400340034003406
:102B30004E34433420343134203420342034203493
:102B4000003400340034003400349C340034003449
:102B50000034003400340034003464340034003471
:102B600000347D348334FF34FF34FF34FF34FF34CA
:102B70004E34433420343234203420342034203452
:102B80000034003400340034003400349C34003409
:102B90000034003400340034003400346434003431
:102BA00000347D348334FF34133410341134123440
:102BB0004E34433420343334203420342034203411
:102BC00000340034003400340034003400349C34C9
:102BD00000340034003400340034003400346434F1
:102BE00000347D348334FF34043405340634073430
:102BF0004E344334203434342034203420342034D0
:102C00009C34003464340034003400340034003424
:102C1000643400349C340034003400340034003414
:102C200000347D348334053456347234743475344E
:102C30004E3461346B346C346F346E3420344C3425
:102C400000349C349C3400340034003400340034AC
:102C5000003464346434003400340034003400340C
:102C600000347D348334FF346C346E3469346B3417
:102C700050347234653464346B346C346F346E3475
:102C800000340034003400340034003400340034A4
:102C90000034003400340034003400340034003494
:102CA00000347D348334FF34203433347834533467
:102CB0004F347434613463346B34793420342034C9
:102CC0000034003400349C340034003400340034C8
:102CD00000340034003464340034003400340034F0
:102CE00000347D348334FF346534723476346F3489
:102CF00056347234743475346C346B34613420342B
:102D000000340034003400349C3400340034003487
:102D100000340034003400346434003400340034AF
:102D200000347D348334FF34003400340034003404
:102D30004E34433420343134203420342034203491
:102D4000643400349C3400340034003400340034E3
:102D50009C340034643400340034003400340034D3
:102D600000347D348334FF34FF34FF34FF34FF34C8
:102D70004E3461346B346C346F346E3420345234DE
:102D80000034003400340034003400349C34003407
:102D9000003400340034003400340034643400342F
:102DA00000347D348334FF3413341034113412343E
:102DB0004E34433420343234203420342034203410
:102DC00000340034003400340034003400349C34C7
:102DD00000340034003400340034003400346434EF
:102DE00000347D348334FF3404340534063407342E
:102DF0004E344334203433342034203420342034CF
:102E00009C349C349C34003400340034003400344E
:102E100064346434643400340034003400340034E6
:102E200000347D348334053456347234743475344C
:102E30004E3461346B346C346F346E344C345034F3
:102E40009C3464349C340034003400340034003446
:102E500064349C346434003400340034003400346E
:102E600000347D348334FF346C346E3469346B3415
:102E70004E3461346B346C346F346E344C345A34A9
:102E800000340034003400349C3400340034003406
:102E9000003400340034003464340034003400342E
:102EA00000347D348334FF34203434347834533464
:102EB0004F347434613463346B34793420342034C7
:102EC0000034003400349C340034003400340034C6
:102ED00000340034003464340034003400340034EE
:102EE00000347D348334FF346534723476346F3487
:102EF00056347234743475346C346B346134203429
:102F000064349C349C340034003400340034003485
:102F10009C346434643400340034003400340034AD
:102F200000347D348334FF34003400340034003402
:102F30004E3461346B346C346F346E3452345034EC
:102F4000643464349C34003400340034003400347D
:102F50009C349C3464340034003400340034003435
:102F600000347D348334FF34FF34FF34FF34FF34C6
:102F70004E3461346B346C346F346E3452345A34A2
:102F8000003400340034003400349C340034003405
:102F9000003400340034003400346434003400342D
:102FA00000347D348334FF3413341034113412343C
:102FB0004E3443342034313420342034203420340F
:102FC0000034003400340034003400349C340034C5
:102FD00000340034003400340034003464340034ED
:102FE00000347D348334FF3404340534063407342C
:102FF0004E344334203432342034203420342034CE
:103000009C34003400340034003400340034003484
:1030100064340034003400340034003400340034AC
:1030200000347D34833400344134753474346F3467
:10303000523469347A3465346E346934203420343F
:1030400000349C3400340034003400340034003444
:10305000003464340034003400340034003400346C
:1030600000347D348334FF34203420342034203441
:103070004E3443342034313420342034203420344E
:10308000003400349C340034003400340034003404
:10309000003400346434003400340034003400342C
:1030A00000347D348334FF34203420342034203401
:1030B00050346C3479346E3420342034203420344D
:1030C0000034003400349C340034003400340034C4
:1030D00000340034003464340034003400340034EC
:1030E00000347D348334FF342034203420342034C1
:1030F0004E344334203432342034203420342034CD
:1031000000340034003400349C3400340034003483
:1031100000340034003400346434003400340034AB
:1031200000347D348334FF34003400340034003400
:103130004E3443342034333420342034203420348B
:10314000003400340034003400349C340034003443
:10315000003400340034003400346434003400346B
:1031600000347D348334FF34FF34FF34FF34FF34C4
:103170004E3443342034343420342034203420344A
:103180000034003400340034003400349C34003403
:10319000003400340034003400340034643400342B
:1031A00000347D348334FF3413341034113412343A
:1031B0004E34433420343534203420342034203409
:1031C00000340034003400340034003400349C34C3
:1031D00000340034003400340034003400346434EB
:1031E00000347D348334FF3404340534063407342A
:1031F0004E344334203436342034203420342034C8
:103200000034833483340034003400340034003418
:1032100000347D347D340034003400340034003414
:10322000DF347D348334203454346F3472346E345C
:103230004C3420346B347234693464342E3420348A
:1032400000347D34833400340034003400340034DE
:10325000003483347D3400340034003400340034CE
:1032600000347D348334FF34613464346F3420346B
:10327000523420346B347234693464342E34203444
:103280000034003400349C34003400340034003402
:10329000003400340034643400340034003400342A
:1032A00000347D348334FF344D3469346E346934F2
:1032B00050346C3479346E3420342034203420344B
:1032C000003400340034003400340034003400345E
:1032D000003400340034003400340034003400344E
:1032E00000347D348334FF342034203420342034BF
:1032F0004334683461346E346E3465346C34343441
:10330000003400340034003400340034003400341D
:10331000003400340034003400340034003400340D
:1033200000347D348334FF340034F3340334003408
:103330004334683461346E346E3465346C343534FF
:1033400000340034003400340034003400340034DD
:1033500000340034003400340034003400340034CD
:1033600000347D348334FF34FF34FF34FF34FF34C2
:103370004334683461346E346E3465346C343634BE
:10338000003400340034003400340034003400349D
:10339000003400340034003400340034003400348D
:1033A00000347D348334FF34133410341134123438
:1033B0004334683461346E346E3465346C3437347D
:1033C000003400340034003400340034003400345D
:1033D000003400340034003400340034003400344D
:1033E00000347D348334FF34043405340634073428
:1033F0004334683461346E346E3465346C3438343C
:10340000003400340034003400340034003400341C
:10341000003400340034003400340034003400340C
:1034200000347D348334003446347234653465347A
:103430004334683461346E346E3465346C34313402
:1034400000340034003400340034003400340034DC
:1034500000340034003400340034003400340034CC
:1034600000347D348334FF3420342034203420343D
:103470004334683461346E346E3465346C343234C1
:10348000003400340034003400340034003400349C
:10349000003400340034003400340034003400348C
:1034A00000347D348334FF342034203420342034FD
:1034B0004334683461346E346E3465346C34333480
:1034C000003400340034003400340034003400345C
:1034D000003400340034003400340034003400344C
:1034E00000347D348334FF342034203420342034BD
:1034F0004334683461346E346E3465346C3434343F
:10350000003400340034003400340034003400341B
:10351000003400340034003400340034003400340B
:1035200000347D348334FF340034003400340034FC
:103530004334683461346E346E3465346C343534FD
:1035400000340034003400340034003400340034DB
:1035500000340034003400340034003400340034CB
:1035600000347D348334FF34FF34FF34FF34FF34C0
:103570004334683461346E346E3465346C343634BC
:10358000003400340034003400340034003400349B
:10359000003400340034003400340034003400348B
:1035A00000347D348334FF34133410341134123436
:1035B0004334683461346E346E3465346C3437347B
:1035C000003400340034003400340034003400345B
:1035D000003400340034003400340034003400344B
:1035E00000347D348334FF34043405340634073426
:1035F0004334683461346E346E3465346C3438343A
:10360000003400340034003400340034003400341A
:10361000003400340034003400340034003400340A
:1036200000347D3483340034463472346534653478
:103630004334683461346E346E3465346C34313400
:1036400000340034003400340034003400340034DA
:1036500000340034003400340034003400340034CA
:1036600000347D348334FF3420342034203420343B
:103670004334683461346E346E3465346C343234BF
:10368000003400340034003400340034003400349A
:10369000003400340034003400340034003400348A
:1036A00000347D348334FF342034203420342034FB
:1036B0004334683461346E346E3465346C3433347E
:1036C000003400340034003400340034003400345A
:1036D000003400340034003400340034003400344A
:1036E00000347D348334FF342034203420342034BB
:1036F0004334683461346E346E3465346C3434343D
:103700000034003400340034003400340034003419
:103710000034003400340034003400340034003409
:1037200000347D348334FF340034003400340034FA
:103730004334683461346E346E3465346C343534FB
:1037400000340034003400340034003400340034D9
:1037500000340034003400340034003400340034C9
:1037600000347D348334FF34FF34FF34FF34FF34BE
:103770004334683461346E346E3465346C343634BA
:103780000034003400340034003400340034003499
:103790000034003400340034003400340034003489
:1037A00000347D348334FF34133410341134123434
:1037B0004334683461346E346E3465346C34373479
:1037C0000034003400340034003400340034003459
:1037D0000034003400340034003400340034003449
:1037E00000347D348334FF34043405340634073424
:1037F0004334683461346E346E3465346C34383438
:103800000034003400340034003400340034003418
:103810000034003400340034003400340034003408
:1038200000347D3483340034463472346534653476
:103830004334683461346E346E3465346C343134FE
:1038400000340034003400340034003400340034D8
:1038500000340034003400340034003400340034C8
:1038600000347D348334FF34203420342034203439
:103870004334683461346E346E3465346C343234BD
:103880000034003400340034003400340034003498
:103890000034003400340034003400340034003488
:1038A00000347D348334FF342034203420342034F9
:1038B0004334683461346E346E3465346C3433347C
:1038C0000034003400340034003400340034003458
:1038D0000034003400340034003400340034003448
:1038E00000347D348334FF342034203420342034B9
:1038F0004334683461346E346E3465346C3434343B
:103900000034003400340034003400340034003417
:103910000034003400340034003400340034003407
:1039200000347D348334FF340034003400340034F8
:103930004334683461346E346E3465346C343534F9
:1039400000340034003400340034003400340034D7
:1039500000340034003400340034003400340034C7
:1039600000347D348334FF34FF34FF34FF34FF34BC
:103970004334683461346E346E3465346C343634B8
:103980000034003400340034003400340034003497
:103990000034003400340034003400340034003487
:1039A00000347D348334FF34133410341134123432
:1039B0004334683461346E346E3465346C34373477
:1039C0000034003400340034003400340034003457
:1039D0000034003400340034003400340034003447
:1039E00000347D348334FF34043405340634073422
:1039F0004334683461346E346E3465346C34383436
:103A00000034003400340034003400340034003416
:103A10000034003400340034003400340034003406
:103A200000347D3483340034463472346534653474
:103A30004334683461346E346E3465346C343134FC
:103A400000340034003400340034003400340034D6
:103A500000340034003400340034003400340034C6
:103A600000347D348334FF34203420342034203437
:103A70004334683461346E346E3465346C343234BB
:103A80000034003400340034003400340034003496
:103A90000034003400340034003400340034003486
:103AA00000347D348334FF342034203420342034F7
:103AB0004334683461346E346E3465346C3433347A
:103AC0000034003400340034003400340034003456
:103AD0000034003400340034003400340034003446
:103AE00000347D348334FF342034203420342034B7
:103AF0004334683461346E346E3465346C34343439
:103B00000034003400340034003400340034003415
:103B10000034003400340034003400340034003405
:103B200000347D348334FF340034003400340034F6
:103B30004334683461346E346E3465346C343534F7
:103B400000340034003400340034003400340034D5
:103B500000340034003400340034003400340034C5
:103B600000347D348334FF34FF34FF34FF34FF34BA
:103B70004334683461346E346E3465346C343634B6
:103B80000034003400340034003400340034003495
:103B90000034003400340034003400340034003485
:103BA00000347D348334FF34133410341134123430
:103BB0004334683461346E346E3465346C34373475
:103BC0000034003400340034003400340034003455
:103BD0000034003400340034003400340034003445
:103BE00000347D348334FF34043405340634073420
:103BF0004334683461346E346E3465346C34383434
:103C00000034003400340034003400340034003414
:103C10000034003400340034003400340034003404
:103C200000347D3483340034463472346534653472
:103C30004334683461346E346E3465346C343134FA
:103C400000340034003400340034003400340034D4
:103C500000340034003400340034003400340034C4
:103C600000347D348334FF34203420342034203435
:103C70004334683461346E346E3465346C343234B9
:103C80000034003400340034003400340034003494
:103C90000034003400340034003400340034003484
:103CA00000347D348334FF342034203420342034F5
:103CB0004334683461346E346E3465346C34333478
:103CC0000034003400340034003400340034003454
:103CD0000034003400340034003400340034003444
:103CE00000347D348334FF342034203420342034B5
:103CF0004334683461346E346E3465346C34343437
:103D00000034003400340034003400340034003413
:103D10000034003400340034003400340034003403
:103D200000347D348334FF340034003400340034F4
:103D30004334683461346E346E3465346C343534F5
:103D400000340034003400340034003400340034D3
:103D500000340034003400340034003400340034C3
:103D600000347D348334FF34FF34FF34FF34FF34B8
:103D70004334683461346E346E3465346C343634B4
:103D80000034003400340034003400340034003493
:103D90000034003400340034003400340034003483
:103DA00000347D348334FF3413341034113412342E
:103DB0004334683461346E346E3465346C34373473
:103DC0000034003400340034003400340034003453
:103DD0000034003400340034003400340034003443
:103DE00000347D348334FF3404340534063407341E
:103DF0004334683461346E346E3465346C34383432
:103E00000034003400340034003400340034003412
:103E10000034003400340034003400340034003402
:103E200000347D3483340034463472346534653470
:103E30004334683461346E346E3465346C343134F8
:103E400000340034003400340034003400340034D2
:103E500000340034003400340034003400340034C2
:103E600000347D348334FF34203420342034203433
:103E70004334683461346E346E3465346C343234B7
:103E80000034003400340034003400340034003492
:103E90000034003400340034003400340034003482
:103EA00000347D348334FF342034203420342034F3
:103EB0004334683461346E346E3465346C34333476
:103EC0000034003400340034003400340034003452
:103ED0000034003400340034003400340034003442
:103EE00000347D348334FF342034203420342034B3
:103EF0004334683461346E346E3465346C34343435
:103F00000034003400340034003400340034003411
:103F10000034003400340034003400340034003401
:103F200000347D348334FF340034003400340034F2
:103F30004334683461346E346E3465346C343534F3
:103F400000340034003400340034003400340034D1
:103F500000340034003400340034003400340034C1
:103F600000347D348334FF34FF34FF34FF34FF34B6
:103F70004334683461346E346E3465346C343634B2
:103F80000034003400340034003400340034003491
:103F90000034003400340034003400340034003481
:103FA00000347D348334FF3413341034113412342C
:103FB0004334683461346E346E3465346C34373471
:103FC0000034003400340034003400340034003451
:103FD0000034003400340034003400340034003441
:103FE00000347D348334FF3404340534063407341C
:103FF0004334683461346E346E3465346C34383430
:00000001FF
